:020000020000FC
:100000007CCEC1C10000000020C000008EC00000F6
:10001000000098C000000000000000000203040679
:10002000080C10182030406080000406080C1018DE
:100030002030406080A0C0000003070F1F000D0D9E
:100040000403060D0503030202004FB662FD0CC057
:10005000552041F00994C52DC095089483FDC7959E
:10006000C4BD64604FBE1895C0916400089483FDC0
:10007000C795C4BD6B7FC0916400CF3F09F41EC01B
:1000800070FF1AC082FD05C04FBE9198909893985A
:10009000189576FD0EC064FD0CC0C091B100C0FD86
:1000A0009498C1FD9798C2FD9598CAEFC095CA95DE
:1000B000F1F79198909893984FBE189524BCCC274F
:1000C000C064C8BF6460F8CFC6CF70FFC4CF64FD02
:1000D000C2CF919AC0CF70FFBECF64FDBCCF909AC3
:1000E000BACF70FFB8CF64FDB6CF939AB4CF949ACD
:1000F00070FFB1CF64FDAFCFC7E0CA95F1F7919A19
:10010000AACF979A70FFA7CF64FDA5CFC7E0CA9585
:10011000F1F7909AA0CF959A70FF9DCF64FD9BCF89
:10012000C7E0CA95F1F7939A96CF4FB6C9B7CF7E7D
:10013000C9BF6E7FCCB5CE0DDDB5DF1DDBBDCABD41
:100140004FBE18953FB68F7EABB7A074A2118061E9
:10015000A0E0ABBFA9B7AE7FA9BF7894A09168001B
:10016000AA2341F085FD2EC0A0916800AA95A09316
:10017000680028C040E050E085FD14C0A0B396FDA3
:10018000A095A2FD4FEFA3E096FDA2E0A5BFAA2790
:10019000A064AABF8D7FA0B396FDA095A2FD5FEFDE
:1001A000451741F7A0E461FDA093680085FD03C0F9
:1001B000A0E4A0936800409396008160442311F06E
:1001C0002092990085FD0EC0A0916900AA2331F00C
:1001D000A0916900AA95A093690004C08061AA2734
:1001E000A064AABF80FF0AC0A09196004A2F61FFB9
:1001F0008E7F85FD01C000C0409361004091B40036
:10020000443009F004C0A0916100A0936300A09164
:100210006000A395A093600051F0F894A9B7A16085
:10022000A9BF84FF02C0A0E4ABBF3FBE1895A09158
:100230007400A395A093740042E050916800552388
:1002400029F085FF03C05A9550936800A09196004D
:10025000A13018F0209299000DC020929A002092AF
:10026000A300A0919900AF5FA093990018F0AFEFA1
:10027000A0939900B09061005091B400523049F4BD
:1002800065FF91F0A2E3BA1678F0A0918600A093E2
:100290006100533049F465FF39F0A2E3BA1620F04B
:1002A000A091C000A0936100509162005B1521F005
:1002B00010F05A9501C05395509362004A95D1F6BB
:1002C0005091A300539509F45A955093A300A0911F
:1002D000A400AA95A093A40009F04BC0A1E0A093AC
:1002E000A40048E0A091A500AA2381F145E0A091D7
:1002F000A5005A17F0F1A091A6005A1728F441E082
:10030000A3E0A093A40007C0A091A7005A1718F477
:1003100041E04093A400D0909C00C0906300DC14A6
:10032000A8F0A091B400A430D9F065FD0FC0C09230
:100330009C00539521F0A091A500A093A300A1E0FB
:10034000A093A400ACE3A093620013C0A0919C0012
:10035000A40F20F45FEF50939C0002C0A0939C0078
:10036000A0919C00AF3F29F4AFEFA0939A00A09317
:10037000A300F894A9B7A160A9BF84FF02C0A0E4BC
:10038000ABBF3FBE18953FB64CB55DB58F7EABB7E2
:10039000A074A2118061A0E0ABBFA9B7AE7FA9BFD6
:1003A000789481FD23C0A2E096FDA3E0A5BF826002
:1003B000A0B396FDA095A2FF05C0409365005093A1
:1003C00066001CC1A3E096FDA2E0A5BFAA27A06419
:1003D000AABF8D7F85FF01C004C140E0A0B396FD98
:1003E000A095A2FDFEC040939600EDC0A3E096FD4F
:1003F000A2E0A5BF8D7F61FF71C0A2E096FDA3E0E2
:10040000A5BFAA27A064AABF826040939100509321
:100410009200A0908F004A19B09090005B09BB2415
:10042000A22C4C38520518F42092950049C0A09196
:10043000D400AA2359F1483C520528F4A0E1BA2E71
:10044000AAE0AA2E23C04836A1E05A0728F4A8E063
:10045000BA2EAFE0AA2E1AC0403DA2E05A0728F4F7
:10046000A4E0BA2EAEE1AA2E11C0403AA5E05A0788
:1004700028F4A2E0BA2EACE3AA2E08C04839A8E0BE
:100480005A0720F4A1E0BA2EA8E7AA2EC42EA09104
:100490009300CA1AD52EA0919400DA0ADD202AF41E
:1004A000AFEFC094D094CA1ADA0A20929500A8E05F
:1004B000A210A0E0CA14DA0618F4A1E0A0939500F7
:1004C000409393005093940040919100509192007A
:1004D00040938F005093900042E075C0A09165005A
:1004E0004A1BA09166005A0B94FD60C093FD5EC04C
:1004F00092FD5AC086FF03C0D52EC42E0CC056955F
:10050000479591FD51C05695479590FD4DC0D52E0C
:10051000C42ED694C79461FD19C0AC2DAC51AD2D3D
:10052000A24008F005C0DD2089F4AC2DA85C70F471
:10053000A0916700A395AA2311F0A0936700AA30A9
:1005400008F44FC02092960081604BC0A0916700D4
:10055000AA2319F0AA95A0936700A22C5091BA0083
:1005600097FD02C0A090C800AAEFAA0EA22DA21D5E
:10057000CA18DA0A4FB74170442319F040E050E03E
:1005800015C0AFEFCA16D20418F04FEF50E00EC0FE
:10059000A091AC00CA9E412D000C441F50E008F011
:1005A00012C04FEF50E00FC05695479594FF07C01B
:1005B000552309F04FEFA42FA6954A0F521D4F3F28
:1005C000520508F04FEF40939600816061FF09C02B
:1005D000AFE1A095A923AB299A2F8F7DBB2009F409
:1005E0008062A0E4A093680085FF03C0AAE0A09306
:1005F000680061FD03C085FD01C08F7E85FD03C0DD
:10060000A0E2A0936900F894A9B7A160A9BF84FFF4
:1006100002C0A0E4ABBF3FBE189511E00AC013E0D2
:1006200008C01AE006C01EE104C014E602C018ECBF
:1006300000C005E1BB27BA95F1F70A95D9F71A95DD
:10064000C1F708952AE338E709C020E33CE806C073
:100650002AE234EB03C025E238EC00C0B091AD00D3
:10066000BA9509F4089512E0BB27979ABA95F1F765
:10067000909ABA95F1F79098BA95F1F79798BA953C
:10068000F1F7123009F0919A123009F4939AB0916F
:10069000AD00BA95F1F7123009F09198123009F4D3
:1006A0009398B7E8BA95F1F71A95F1F6022FB22FA1
:1006B000BA95F1F70A95D9F73A9581F6979A089580
:1006C000221B39E0001F3A9509F40895221F211BCF
:1006D00018F4210F8894F6CF0894F4CF622C722C72
:1006E000B0E08894B395221F331FE0F73795279524
:1006F0008894912E802E020B130B10F4192D082DC7
:1007000010F4889401C00894661C771CBA9571F7A0
:10071000172D062D0895322D11232AF43A950095B0
:100720001095031B130BF894029F712C002D129F40
:10073000912C802C7894780C172D921C292DB4E0E4
:100740006B2E2695179507956A94D9F7332321F0D8
:1007500000951095031B130B08950091B40004300D
:1007600009F474C0B0919600B95198F0B72FB670E3
:1007700081F465FD2BC005E09090C600B92DBA95B7
:1007800021F00AE0BA9509F002E1B0917B00B01BBC
:10079000E0F065FF0AC0B0919E00B0939C00BFEFEF
:1007A000B093A300B1E0B093A400B0916100B09306
:1007B000630020927E0020927F0020928000209291
:1007C0008100209282006F7D41C060629090C600DF
:1007D000B92DBA9579F4B0916200B095BB1FBB1FDB
:1007E0001B2FB7950B2FB12FB170B3951B2FB02FC7
:1007F000BE7F25C0B92DBA95BA9581F4B09162003B
:10080000B095BB1FBB1FBB1F1B2FB7950B2FB12F65
:10081000B370B3951B2FB02FBC7F14C0B091620092
:10082000B095BB1FBB1FBB1FBB1F1B2FB7950B2F4B
:10083000B12FB770B395B3951B2FB02FB87FB054BD
:100840000B2F120900937E0010937F0008951091E2
:100850007B00169500917A000795B0917E00B01B41
:100860000B2FB0917F00B10B1B2F28F40038BFEF86
:100870001B0740F009C00F37120508F405C00FE749
:1008800010E002C000E81FEF009383001093840083
:10089000089500918300B09180000B0F10918400A7
:1008A000B09181001B1F20E03091840033230AF4B3
:1008B0002A95B09182002B1F1AF4203F40F00AC005
:1008C0002F3008F407C00FEF1FEF2FE003C000E048
:1008D00010E020EF30916300B0919B003B1718F4BB
:1008E000323030F009C0B0918400BB235AF004C00C
:1008F000B0918400BB2332F40093800010938100F8
:100900002093820008952091D70000918300000F6A
:1009100010918400111FFFDE11232AF40038BFEF6D
:100920001B0740F009C00F37120508F405C00FE798
:1009300010E002C000E81FEF002352F0B091620007
:10094000B01B0B2F18F0013008F00AC001E008C0FE
:1009500000950F5FB09162000B0F08F001C00FEF20
:100960000093850008952091D80000918100109196
:100970008200D1DE11232AF40130BFEF1B0740F0C3
:1009800009C00F3F120508F405C00FEF10E002C0C8
:1009900001E01FEF112352F0B0918500B01B0B2F27
:1009A00018F0013008F00AC001E008C000950F5FA0
:1009B000B09185000B0F08F001C00FEF00936300AA
:1009C00008950FEF71FD1EC0B091D300BB23D1F08D
:1009D000B0917B00BB23B1F00FEF10917B0070DE74
:1009E000F894B091730072FDB5E00B9F112D002DAE
:1009F0007894112309F00FEFB0919E000B1710F4BB
:100A000000919E0000939D00089500917A0010913E
:100A10007B0000541140B0919D0010F4BA9501C0C4
:100A2000B39511F0B0939D000895F0D3B7E074FD35
:100A3000B7E0B06CB7B9B6B1B068B064B6B9EDDDC7
:100A4000B7E074FDB7E0B06CB7B9B6B1B068B064E8
:100A5000B6B9B6B1B6FDFDCF04B115B1B6B1BF7729
:100A6000B6B92BD420E02093A800222309F441C07A
:100A700030E03093A900732E7694622E6694620E55
:100A8000731E262D372D0217130778F08090A800CB
:100A9000B0E0B80DB093A8008090A900B0E0B81DF8
:100AA000B093A900260D371DEECF8090A80090903E
:100AB000A9001091A90016950091A8000795169518
:100AC000079523E0169507952A95E1F72091B50043
:100AD0002A9529F42092A8002092A9000AC02A95FC
:100AE00021F0800E911E2A95E1F78092A800909245
:100AF000A90008952091B500B6B1B6FDFBCF04B1B1
:100B000015B1B6B1BF77B6B9B091AA00B395B0939D
:100B1000AA00B83060F12092AA00B091D200BB23A5
:100B200021F1112329F0B091AB00BF3F61F009C062
:100B3000B091AB000B1739F020F4BB2321F0BA952C
:100B400002C0B395E1F300919B00B093AB00B030CD
:100B500050F400ECB03038F400E8B03020F400E499
:100B6000B03008F400E000939B007F7E08952130B0
:100B7000B1F00F3FB3E01B0790F4B0E0BB2379F076
:100B8000B091A8000B17B091A9001B0740F4B091D9
:100B90009B00BB2359F0BA95B0939B0007C0B0915E
:100BA0009B00BF3F19F0B395B0939B0000919B0051
:100BB000B0916300B01B10F400916300B0919C00F1
:100BC0000B1750F000919C00B0919C00BF3F21F0AA
:100BD000B0919C00B0939B00502E00936400B091A4
:100BE000AA00B73009F47061089502E3F894B09157
:100BF000D9000B9F012D000C001F7894B0919B0031
:100C00000B1710F000919B000093610000936300AC
:100C1000502E0093640000939E00089520927A0065
:100C2000B0EFB0937B000895F8940CB51DB52091FA
:100C30007400789430917500609076000093750090
:100C400010937600031B160971FD03C077FD80C069
:100C500028C070907700209377002709222319F08D
:100C60000FEF1FEF0EC080907800909079003093C6
:100C70007800609279000091750010917600081953
:100C8000190920917A0030917B0036952795020F43
:100C9000131F10F40FEF1FEF00937A0010937B00E7
:100CA0002BC020917A0030917B003901B4E08B2E6B
:100CB000B2E09B2E343040F08A949A94383020F081
:100CC00072FD02C08A949A94769467948A94E1F7AC
:100CD00026193709992021F0169507959A94E1F77E
:100CE000200F311F20937A0030937B0028F43FEFD0
:100CF00030937A0030937B00323008F4706871FFD3
:100D000002C0B3E00DC0B091C40000917100023880
:100D100038F0B395003A08F0B395B63008F0B5E076
:100D20009B2EB4E08B2E10917B0000917A0024E082
:100D3000169507952A95E1F70819120928F0B02FA2
:100D4000B250B12FB20910F402E010E0980126C0B1
:100D500020917A0030917B003901769467946694F3
:100D6000669466942619320906950695200F321D61
:100D700020937A0030937B00323008F07F7704E0D4
:100D8000369527953695279526952695201B10F0A4
:100D9000223008F422E089019090C40060FDFECF6B
:100DA000E0908B00F0908C006160B9B7B061B9BF82
:100DB000380177FD41C07694679400938B001093BF
:100DC0008C00B92DB330E1F0B0FD04C0060D171D45
:100DD000930106C0000F111F0250120922E030E0FB
:100DE000B92DB33068F020938D0030938E000093BE
:100DF0008700109388006092890070928A003AC040
:100E000000938D0010938E0020938700309388000C
:100E10006092890070928A0071FF0DC0BFE0B093AC
:100E20008D0020928E00B093890020928A00B093AA
:100E30008B0020928C001EC0669400938B00B92D0D
:100E4000B33091F0B0FD03C0060D262D03C0000F96
:100E5000025022E0B92DB33038F020938D0000937A
:100E600087006092890006C000938D002093870060
:100E70006092890000917C0002FD0350013031F442
:100E800095FD0CC0B2E0B06CB7B90BC0023021F4D4
:100E9000B3E0B06CB7B905C095FDF4CFB4E0B06C69
:100EA000B7B90091A200000F10F4BBE60B27009326
:100EB000A20060FDFECFB2E0B0936E006160B9B7F2
:100EC000B061B9BFB72FB670D1F020917A003091E0
:100ED0007B00369527953695279571FF02C0B0E4C3
:100EE0003B0FF8940CB51DB5020F131F1BBD0ABDB7
:100EF0006160B0E1B8BFB9B7B061B9BF7894089587
:100F0000686020927D0020E066FD20E206C06860F7
:100F100020927D0020E266FD20E001E011E077FDF7
:100F200011C0B72FB67009F0677F14E100917B0004
:100F3000069509F403950F3008F00FE071FF02C029
:100F400004E114E160FD0FC0B0917D00BB2359F0B6
:100F500071FF06C0B0916E00BA95B0936E0011F4A7
:100F600070624FC0ABDFB0B7B77FB0BFB8B1B0B73A
:100F7000B860B0BFB0917D00B395B0937D00B8B1BB
:100F800077FD06C0B1E071FDB3E0BA95F1F7B8B1F5
:100F9000B072B21709F02AC071FF05C0039501179E
:100FA00008F00A95CFCF63FD05C00395011708F03F
:100FB000B4CFC8CF677FF8943CB56DB470907A0019
:100FC000B0917B00770CBB1F08F4BFEF770CBB1F01
:100FD00008F4BFEF370D6B1E6BBC3ABD6160B0E12A
:100FE000B8BFB9B7B061B9BF789497CFB0916D0071
:100FF000B13008F492CF63FD90CF0A9509F0A2CFEB
:101000007F7D20918D0030918E00F894B0E1B8BFC3
:101010000CB51DB5020F131F1BBD0ABDE090870064
:10102000F09088006160B9B7B061B9BF7894B72F0C
:10103000B67039F0B0916D0072FFB395B0936D004A
:1010400009C075FF07C066FD05C063FD03C0BF9101
:10105000BF91FAC4089500E063FF01C001E0F89475
:1010600010917100B7E01B9F212D102D7894200F57
:101070002695179526951795269517951093710027
:10108000183718F4B8E7B093710000917100B0916F
:1010900072000B1720F0606191989098939860FD12
:1010A000FECFE0908900F0908A006160B9B7B0612E
:1010B000B9BF0895B2E095FD0AC0F894B0937C00E2
:1010C000979A949862FF01C0939A7894F4C0F89428
:1010D000B0937C00979A959862FF01C0919A78949A
:1010E000EAC0B3E082FF24C095FD11C002E0F8948D
:1010F000B0937C00E1E8F0E00093B1009398959AFA
:1011000062FF02C0909A01C097987894D4C002E020
:10111000F894B0937C00E1E8F0E00093B10091987E
:10112000949A62FF02C0909A01C097987894C3C0C5
:1011300095FD0BC0F894B0937C00EBE6F0E093983B
:1011400062FF01C0909A7894B6C0F894B0937C0086
:10115000EBE6F0E0919862FF01C0909A7894ABC002
:10116000B4E095FD0AC0F894B0937C00949A9598E9
:1011700062FF01C0909A78949EC0F894B0937C006E
:10118000959A949862FF01C0909A789494C0B5E0C3
:1011900082FF24C095FD11C001E0F894B0937C005B
:1011A000E7E7F0E00093B1009098979A62FF02C0E1
:1011B000919A01C0949878947EC004E0F894B0931A
:1011C0007C00EBE8F0E00093B1009098979A62FF02
:1011D00002C0939A01C0959878946DC095FD0BC09C
:1011E000F894B0937C00E5E6F0E0909862FF01C0CF
:1011F000919A789460C0F894B0937C00E1E7F0E0B5
:10120000909862FF01C0939A789455C0B6E095FD1E
:101210000AC0F894B0937C00959A979862FF01C039
:10122000919A789448C0F894B0937C00949A9798D7
:1012300062FF01C0939A78943EC0B1E082FF24C05F
:1012400095FD11C004E0F894B0937C00EBE8F0E069
:101250000093B1009198949A62FF02C0939A01C0E2
:101260009598789428C001E0F894B0937C00E7E763
:10127000F0E00093B1009398959A62FF02C0919AB2
:1012800001C09498789417C095FD0BC0F894B09362
:101290007C00E1E7F0E0919862FF01C0939A7894B6
:1012A0000AC0F894B0937C00E5E6F0E0939862FF02
:1012B00001C0919A78946F7E089524E630E0F90198
:1012C0002092B100919890989398949A979A959AB1
:1012D0006B7F0895A2EBB0E007E00D9307E00D935C
:1012E00001E00D9304E00D930FEF0D930D9309E0D2
:1012F0000D9302E00D9301E00D9301E00D93AEEB31
:10130000B0E001E00D9300E00D9304EB0D930FEFBF
:101310000D930D930D9303E00D930FEF0D9301E0EB
:101320000D930FEF0D9305E20D9300ED0D9308E77C
:101330000D9308EC0D9304E00D930FEF0D9301E076
:101340000D9300E00D930AE70D930AE00D9300E082
:101350000D9301E00D9300E00D930FEF0D9300E06E
:101360000D9308952091B9008B7F233009F4846098
:10137000B091BA009F7DB1FD90629F7BB091BB00A0
:10138000B1FD9064223011F0886001C0877F08951C
:101390000A95E00FF21DB4910895ECE1F0E00091A0
:1013A000B200F6DFB093D700ECE1F0E00091B300BB
:1013B000EFDFB093D800EAE2F0E00091B800E8DF98
:1013C000B093D9000091D100002319F42092A50018
:1013D00013C0013108F001E1B02FB00FB00FB0938E
:1013E000A5001B2FB10FB10FB00FB093A600B10F26
:1013F000B00FB00FB093A7000091B800023008F40E
:1014000002E000937300B091CE000FEFB23009F408
:1014100000EAB33009F402E800937200E8E3F0E078
:101420000091D500B5DFB093A000089508952091F4
:10143000C8003091C900B091BA00B33009F43E50F1
:1014400097FF02C020E03FEFB32FB21B6B2EB258C4
:1014500010F4B2E86B2E00E00395609EB12DBD57ED
:10146000D8F30093AC0008959068E1DFDCD8DBD8B6
:1014700020E030E0B0E16B2ED2D8B09196002B0F77
:10148000321D6A94C9F7B4E036952795BA95E1F70D
:10149000822E9F77CCDF0895F894E3E0F0E0B9E086
:1014A000B7BFB491B078C1F3F894A895B1B5B8615D
:1014B000B1BDB0E0B1BDB4E0BEBFBFE5BDBFFDDEB4
:1014C000B0E0B8BBB0E1B7BBB0E0B5BBB0E0B4BB17
:1014D000B0EBB2BBBBEBB1BB2224A0E0B0E02D92DD
:1014E000AA31E9F7A0E6B0E00FEF2D920A95E9F7EF
:1014F000B1E0B093A200EEDEE8D2B7E0B06CB7B9CD
:10150000B6B1B460B068B6B90091CA000093AD003E
:10151000B1E0B0936A00F8948AD894D884D895D86A
:1015200082D896D880D860D382D881D87ED8F894D3
:101530000AEF1AEFA0B396FDA095A2FF1FC01A955F
:10154000C9F70A95B1F7E0E0FCE1B591B43E39F492
:10155000B591B03E21F4B591BF3F09F40CC0E0E075
:10156000F395F395B591B83F49F4B591B43931F499
:10157000B591BA3A19F4EE27F6950994F3DE0DDF2A
:1015800055DF55DF0091CA000093AD0096DEB2E052
:10159000B3BFB2E0BEBDB2E0B5BDB1E5B8BFB9BF43
:1015A000B0B7B77FB0BFB8B1B0B7B860B0BF35D8CB
:1015B00078943BDA20927000B3E096FDB2E0B5BFBC
:1015C000B0E4BBBFBB27B064BABF8D7F30D86260C8
:1015D00033E02CE0B0919500BB2321F42CE03A9548
:1015E00009F4A5CF20D880FFA2CF8E7FB0919600BE
:1015F000B23078F3B92FBF71009198000093970033
:10160000B0939800B01729F72A9521F76D7FB3E0C2
:1016100096FDB2E0B5BFBB27B064BABF8D7FB09175
:10162000D400BB2321F48062B92FB0709B2F8F7B35
:1016300020926700FAD785FF05C0B0916700BA30E5
:1016400008F08064ECD702E085FF01C000E0B091B3
:101650009600B017B8F3F894F5D7F4D7F3D7789489
:10166000E6D720928600DBD7B091BE00B13008F4F7
:1016700078C0B0916A00B13008F473C085FD18C01D
:10168000B0919600BF3F08F46CC0F894E4D778940A
:10169000CCD7B0919600B130C0F7F894D3D7C1D76A
:1016A000D1D77894C2D7B0919600BF3FB0F3CEC2E5
:1016B000B8E09B2E9068F894BADE7894B6D7F89488
:1016C0009F77B5DE80909600B0919600BF377894F2
:1016D00008F44FC0A2D7F894BED778949A9451F7E3
:1016E000C3DEB82DB550B093C900A1D7F89481D20C
:1016F0007894BAE09B2E9068F89499DE789495D708
:10170000F8949F7794DE80909600B0919600BF3752
:10171000789478F782D7F89495D783D793D778942D
:101720009A9449F7A1DEB82DBB5FB093C8000B2F88
:101730001091C900125810F0100B20F4B2E80B0FF2
:101740000093C90074D7F894EDD162D278946DD724
:10175000F8946DDE7894B0919600BF3F08F48ECF78
:1017600075C200919600B09186000B1710F000939F
:1017700086005BD701E0B091BA00B35009F405E0F0
:10178000B0919600B01708F06ECFF89464D763D785
:1017900062D778944CD720926A0020926B002092F6
:1017A0006C00B0916B00B395B0936B00BF3F71F5C7
:1017B000B0916C00B395B0936C00B091CC0009E18E
:1017C000BA9559F002E3BA9541F00DE7BA9529F0C0
:1017D0000AEFBA9511F020926C00B0916C00B0172E
:1017E000A8F06BDD1AD7B0916C00BA95B0936C007D
:1017F00020926B00B091CB00B093AD00F8942BD742
:101800007894B091CA00B093AD000FD70AD7B091C9
:101810006800BB2319F485FF01C089CE01E085FD76
:1018200001C006E0B0919600B01708F4BACFFDD61B
:10183000B0916800BB2309F47ACEF8943EDD209283
:1018400061002092620020926300522C209264007A
:101850002092A1007894B091B700BB0FB0939F0085
:1018600020927E0020927F002092800020928100B2
:10187000209282002092AA0060E070E02092710025
:10188000B8E0B093AA007061C8D6B7E074FDB7E0C5
:10189000B06CB7B9B6B1B068B064B6B9B6B1B6FDA0
:1018A000FDCF04B115B1B6B1BF77B6B9112309F0B8
:1018B0000FEF0093AB001ED9B8E0B093AA0070619F
:1018C00051DDF894BFEFB0939B008FD9B0916100C8
:1018D000B0939B00B0939C00B0939D007894B1E0CE
:1018E000B0936100B09363005B2EB0936400B0933B
:1018F000A400B0919A00B093A300B091BA00B330A5
:1019000019F49F7D87FD90627160726020926D0076
:101910007DDC93DC83D988D981D986D97FD9F7DA60
:101920001CD799DBC7DB80D9EBDA65FD90D777FF51
:1019300048D877FD6AD88FDBD4DB76D9E8DA65FD45
:10194000A8D789DB0DDC70D9DBDA65FDDCD783DB5A
:101950001EDC6AD9DCDA65FD06D87DDB57DC64D98C
:10196000CFDAB7E074FDB7E0B06CB7B9B6B1B06824
:10197000B064B6B970DB61DC57D9BCD871FF1EC04A
:10198000B0919E00B0939B00B0939C00B0919A00E0
:10199000B093A300B1E0B093A40018E12CE0B091A3
:1019A0006D00B11728F07D7F746020936F0006C032
:1019B000B0919600B13008F0B2CF50C072FF15C0A0
:1019C00066FD13C0B0916F00BA9519F47B7F786003
:1019D000A6CFB0936F00B0919600B13008F09FCFC2
:1019E000B091BA00B33009F039C020927000B091C4
:1019F0009900B13058F0B0919E00B0939C00B09126
:101A00009A00B093A300B1E0B093A400B091990004
:101A10000AEF1091D600112309F003E0B01708F087
:101A20001DC085FF04C0B0916800BB23B9F000EF72
:101A300066FF05C0B0919E00B0939B0000E2B0919C
:101A40007B00B01708F46BCFB0917000B395B093E2
:101A50007000B0919600BB2309F002C02092700084
:101A6000F8942BDC8090B900B2E0B093B9007ADC36
:101A70008092B9002092610020926200209263005F
:101A8000522C2092640020929F0060E070E07894D5
:101A9000CCD513DC0091D600002319F0919A909ACE
:101AA000939AB7E0B06CB7B9B6B1B460B068B6B9E4
:101AB00085FF05C0B0916800BB2309F438CDB09113
:101AC000BF00B13008F0BECD68CEEDE0F0E023D02D
:101AD000053A09F01BC0EEE0F0E01DD00A3509F030
:101AE00015C03AE0A2EBB0E0E3E0F0E014D00D93D3
:101AF00031963A95D9F739E1AEEBB0E0EFE0F0E09E
:101B00000AD00D9331963A95D9F702C0E3DB0AD09B
:101B1000E8E2F0E00895E199FECFEEBBFFBBE09A6A
:101B20000DB308951ED03AE0A2EBB0E0E3E0F0E0A0
:101B30000D910FD031963A95D9F739E1AEEBB0E07F
:101B4000EFE0F0E00D9105D031963A95D9F712D03B
:101B50000895E199FECF0DBBEEBBFFBBE29AE19A7F
:101B60000895EDE0F0E00FEFF4DFEEE0F0E00FEFCE
:101B7000F0DF0895EDE0F0E005EAEBDFEEE0F0E005
:101B80000AE5E7DF08953091AE000091AF003130F3
:101B900011F40093B200323011F40093B3003330EB
:101BA00011F40093B400343011F40093C6003530C2
:101BB00011F40093B500363011F40093B8003730BB
:101BC00011F40093C400383011F40093B900393097
:101BD00011F40093CE003A3011F40093BA003B3078
:101BE00011F40093BB00089525E021D52A95E9F76B
:101BF000089528D52AD52CD52ED513D523D525D56E
:101C000027D529D50ED51ED520D522D524D5089582
:101C100022D51ED51AD516D504D51DD519D515D55D
:101C200011D5FFD418D514D510D50CD508958090B2
:101C3000AE009090AF0006D505D504D5F2D48A94B5
:101C4000D1F709D5EED49A94E1F70895F894D1DF4D
:101C50007894CADFC9DFB1E0B093AE00B1E0B093D1
:101C6000AF002092B000F894E2DF7894B5E06B2EDC
:101C700070909600DCD4B09196007B16C9F7B13015
:101C800018F0BF3F40F107C07EDFF8944BDFB1DFB3
:101C9000B8E0B1BDA9DF6A9459F7B091B000B3952F
:101CA000B093B000B33008F4DECF9EDFB091AF0048
:101CB000B395B093AF00F894B091AE00BA95EEE34F
:101CC000F0E0EB0FF21D049178940395B091AF0012
:101CD000B01708F4C6CF88DF87DFB091AE00B395A8
:101CE000B093AE00B091AE00BC3008F4B7CFF2DADA
:0C1CF000F89418DFB8E0B1BD77DFCECB70
:00000001FF
